:060000008A150A16612DAD
:020008000800EE
:100020008A150A1600208A110A12F825F012F21217
:10003000DF01E0018611701183120313F801F90149
:10004000FA01FB01FC01FD01FE01FF0120308400EB
:100050000221A000243020020319BA293C302002DA
:10006000031D2828840AD4010230DC000221D407B1
:10007000D8208000840ADC0B36282208D300210E09
:10008000D30406305302DC000221D407D8208000BC
:10009000840ADC0B44280230DC000221D8208000D6
:1000A000840ADC0B4D280221DB003E305B02031D7D
:1000B000802884030008DB008403000EDB0454085E
:1000C0005B02031D89288313243084000008D500B7
:1000D0008403000ED504D50803197D284E3055023F
:1000E00003187D2806118615903055070730031830
:1000F000013E8A00550890271A280030DE00982813
:100100000130DE0098280230DE0098280330DE003F
:1001100098280430DE0098280530DE009828063044
:10012000DE0098280730DE0098280830DE00982886
:100130000A30D3000030D5008317103084005E08E9
:1001400080000615701551211A2841346C346C3426
:10015000203459346F34753472342034423461346D
:10016000733465342034413472346534203442347D
:1001700065346C346F346E346734203454346F34E7
:06018000203455347334F5
:100190003D3081000B110800D83081000B110800A0
:1001A000F63081000B110800EC3081000B110800C3
:1001B000F700F6000F30F605473077020318E628FF
:1001C00041307702031CE6280930F607760808005C
:1001D000CC00CD00F030CD054D0EF420CD000F3019
:1001E0004C05F420CC000800F6000A307602031C0F
:1001F000FC2837307607FE28303076070800F01CE0
:1002000013293829F01C0529212983120313F01A18
:10021000112906148316891B0E290B298312061037
:10022000080806100800F01A202983128C13880091
:1002300006148316091B1A2983128C1F1D29061008
:100240000800831203138C1A292986128C1A292973
:1002500026291A0833291819312998183129030138
:100260003329181218168616CE01CE0B3529080030
:10027000D2000C1E3929520899008316981C3E2979
:10028000422983128312080004305302D0008313E2
:1002900021308400D4010008D407840AD00B4B29F4
:1002A00008008313203084005B308000840A5308E8
:1002B000E8204D088000840A4C088000840A550814
:1002C000E8204D088000840A4C088000840A701DD4
:1002D000862908305302D0000310D00C2530D100FD
:1002E00083171030F7008317770884000008E82090
:1002F0008313510884004D088000D10A840A4C08F9
:100300008000D10A8317F70AD00B732944210330E8
:100310005302F6002030760784005408E8204D0888
:100320008000840A4C088000840A5D3080005308F5
:10033000D0008313203084000008FF20840AD00BF3
:100340009C290800831203138616831640309900F7
:10035000831218121A081A081816080083120313B9
:100360008616831615309900831218121A081A0877
:10037000181608000530DC002130840002218000BE
:10038000840ADC0BBE29DB000D305B02031D7D28D7
:100390003030FF203230FF201A280E30D3000130D9
:1003A000D5008A110A1600208A110A1270155121EF
:1003B00008001230D3000230D500092670155121F3
:1003C00008000E30D3000430D50070150230D8007C
:1003D0008A150A1607208A110A12711CF2290730A1
:1003E000DE007E257015512108000830D30005304D
:1003F000D50083132608DB00250EDB04DB08031978
:10040000022A042A1027052A09275121080008304A
:10041000D3000630D5002608E100250EE1042808A7
:10042000E200270EE2042908E3002A0EE30451212A
:1004300008000A30D3000730D5008A110A160C20B4
:100440008A110A127015512108000A30D3000830B1
:10045000D5004F267015512108000830D30009300F
:10046000D5002608E000250EE004512108000830E0
:10047000D3000A30D5002608DB00250EDB04F2127B
:10048000DB080319442AF2165121080083120313D2
:10049000F016061008000830D3001230D5005121A4
:1004A00008000830D3001B30D5008A110A16AA2193
:1004B0008A110A120430D8002B2508000830D30016
:1004C0001E30D5008A110A16AA218A110A12033099
:1004D000D800002508000830D3002130D5008A114B
:1004E0000A16AD218A110A120930D8000025080029
:1004F0000830D3002230D5008A110A16AD218A11A6
:100500000A120A30D8002B2508000830D300233007
:10051000D5008A110A16B0218A110A121C30D8009F
:10052000002508000830D3002430D5008A110A16AF
:10053000B0218A110A121D30D8002B25080008307E
:10054000D3002530D50051218A110A16E0218A11E5
:100550000A1208000830D3002630D5008A110A1686
:1005600088218A110A12512108000830D30027304F
:10057000D5008A110A168B218A110A12512108000E
:100580000830D3002830D5008A110A16E0218A11DC
:100590000A125121F22C0830D3002930D5008A11DB
:1005A0000A1679218A110A12512108000830D30055
:1005B0002A30D50083132608DD00250EDD048A11BC
:1005C0000A16B3218A110A12512108000830D300FB
:1005D0002B30D5002608DB00250EDB0400305B0243
:1005E0000319FD2A01305B020319152B02305B024F
:1005F0000319FB2A2A2BCF262A2BCF26C8200B1D16
:10060000FF2ABC26C8200B1D032B012787192A2B84
:10061000F926871587110127C82087192A2B0B1D5A
:100620000D2B0730DE007E252A2BCF26C8200B1D80
:10063000172BBC26F9268715871101271930D800FA
:100640008A150A1607208A110A12711C2A2B0730F4
:10065000DE007E25512108000A30D3002C30D50061
:100660000708DB000730DB0503305B020319402B72
:1006700005305B020319422B0030D5000330502BAC
:100680000230502B0127871D4E2B5030DC00871D78
:100690004E2BDC03031D472B0030502B0130502B19
:1006A000DB00831710308400831203135B08800083
:1006B000701551210800CF26C8200B1D5D2BBC26CC
:1006C0000830D3002D30D500512108000830D30068
:1006D0002E30D500F9268715D4200B1D6D2B8711E0
:1006E000C8200B1D712BC8200B1D742BC8200B1D9F
:1006F000772BC8200B1D7A2B0127512108000830C9
:10070000D3002F30D5001A30D800EC2D0830D3009C
:100710003030D5001930D800EC2D0830D3003330FC
:10072000D5002608DB00250EDB0400305B02031D2C
:100730009B2BCF26AA2B01305B02031DA12BBC26CD
:10074000AA2B02305B02031DA72BA926AA2B063079
:10075000DE007E25512108000A30D3003430D50058
:100760008317103084006E26831203131E08831231
:1007700003178000831203137015512108000A30FB
:10078000D3003530D500831710308400A9266A269F
:10079000CF26831203131E088312031780008312CF
:1007A00003137015512108000A30D3003730D500EB
:1007B0008317103084007226831203131E088312DD
:1007C00003178000831203137015512108000830AD
:1007D000D3003930D500A9258A150A16A1208A111F
:1007E0000A12F11CF62B70160730DE00B525080042
:1007F0000830D3003B30D5002508DB0001305B0218
:100800000319062C0630DE007E25102C8A110A16EC
:10081000A7218A110A12711D102C0730DE007E25D7
:10082000512108000830D3003C30D500F801F9010F
:10083000FA01FB01FC01FD01FE01FF018A150A1608
:10084000A1208A110A120127871D232C2A2C073088
:10085000DE007E25512108001030D3003D30D50048
:1008600070150D30D800EC2D0830D3003E30D50087
:100870008A258A110A16E0218A110A1293258A1103
:100880000A1208000830D3003F30D500A9258A118C
:100890000A16E0218A110A12B52508000830D30093
:1008A0004030D5008A258A110A1631218A110A1290
:1008B000932508000830D3004130D500A9258A11BE
:1008C0000A1692208A110A12B52508000830D300B2
:1008D0004230D5005C258A110A16A7218A110A1216
:1008E000512108000830D3004330D500A9258A11D2
:1008F0000A1612208A110A12B52508000830D30002
:100900004430D500A9258A110A1634208A110A120A
:10091000B52508000830D3004530D500A9258A1137
:100920000A1671208A110A12B52508000830D30072
:100930004630D500A9258A110A164F208A110A12BD
:10094000B52508000830D3004730D5008A258A1124
:100950000A16AE208A110A1293258A110A1208007B
:100960000830D3004830D5008A258A110A16D320D2
:100970008A110A12932508000830D3004930D500A7
:100980008A258A110A1612218A110A129325080053
:100990000830D3004A30D5008A258A110A16F32080
:1009A0008A110A12932508000830D3004B30D50075
:1009B0002608DF00250EDF04512108000830D3008F
:1009C0004C30D5005121C8200B1DE42CA221080079
:1009D0000830D3004D30D5005121C8200B1DEE2C1E
:1009E000AE2108000030DE000A30D3000030D50010
:1009F0008317103084005E088000701551210800B4
:100A00005C258A150A1607208A110A12711C0C2D02
:100A10000730DE007E25292D5121D0200B1D0E2D03
:100A20007B30FF20D0200B1D132DD4018A150A1610
:100A30006D218A110A125408E8204D08FF204C0845
:100A4000FF20D0200B1D222D7D30FF20D0200B1D3C
:100A5000272D512108005C258A150A1607208A11C6
:100A60000A12711C372D0730DE007E255A2D5121C8
:100A700002217B3C0319402D0130DE007E255A2DDA
:100A8000D4018A150A1684218A110A120221D8205B
:100A9000DB00DB0E0221D8205B0454020319532D26
:100AA0000430DE00701602217D3C03195A2D0130FE
:100AB000DE007E255121080083132C08F8002B0E40
:100AC000F8042A08F900290EF9042808FA00270E6C
:100AD000FA042608FB00250EFB043408FC00330E44
:100AE000FC043208FD00310EFD043008FE002F0E1C
:100AF000FE042E08FF002D0EFF0408000A30D3006C
:100B00000030D50070158317103084005E08800017
:100B1000061508005C255121D0200B1D8D2D7B3042
:100B2000FF20D40108005408E8204D08FF204C089D
:100B3000FF207D30FF20F11EA72D0A30D3000030AA
:100B4000D50070158317103084005E088000512195
:100B5000080070125C25512102217B3C0319B32D42
:100B60000130DE007016D40108000221D820DB001D
:100B7000DB0E0221D8205B0454020319C22D04307D
:100B8000DE00701602217D3C0319C92D0130DE0004
:100B9000701603138312701ED72D0A30D300003055
:100BA000D50070158317103084005E088000512135
:100BB0000800E8204D08D407FF204C08D407FF2088
:100BC00008000221D407D820CD00CD0E0221D40781
:100BD000D820CD044D0808008A150A1607208A116E
:100BE0000A12711CF62D0730DE007E255121080007
:100BF0008316D0308700A0000514851485150430B5
:100C00009F00831280309F00CF268030E6007E2632
:100C1000080086157208E500DB268A110A16B32142
:100C20008A110A1283120317103084002D26840AB9
:100C30004326840A4626840A4926840A4C2603133E
:100C400083126508F2007218A926F218BC267219E0
:100C5000CF26F219DB2686110800831780010313C3
:100C600083126E2633301E02031C3B2E9A301E0266
:100C700003183F2E422E831701308000422E831727
:100C800080308000080083178001080083178001EE
:100C90000800831780010800831780010800E7011E
:100CA0008317103084008316861506158312CC2016
:100CB0000B1D582E061D5E2E0F30E704861D622E7A
:100CC000F030E70467088317800083168611061149
:100CD000831208009F121F129F11762E9F121F125F
:100CE0009F15762E9F121F169F15762E17271F14FD
:100CF00017271F151F197A2E1F1008008610113094
:100D0000E40088266608E400882686141B2708006D
:100D10000830CF00E40D031C8F2E8617902E86130B
:100D200000000000000000000617000000000000A6
:100D300000000613CF0B8A2E0800861406178617AC
:100D400008008614061786130800861406178613F3
:100D500008000708EA006A15EA146A106A088700A2
:100D60007214F2107211F2118A110A12C8208A113B
:100D70000A120B1DB92E08000708EA006A15EA10CE
:100D80006A146A0887007210F2147211F2118A1143
:100D90000A12C8208A110A120B1DCC2E080007085F
:100DA000EA006A11EA146A146A0887007210F210E5
:100DB0007215F21108000708EA006A15EA146A14AD
:100DC0006A0887007210F2107211F215080094126E
:100DD00083162016A01220088700831285160800AB
:100DE000941283162016A0162008870083128512FD
:100DF000080094128316A01120088700831205159D
:100E0000080094128316A01520088700831205118C
:100E10000800051281010B110B1D0C2F7212080026
:100E2000051681010B110B1D132F72160800CE0140
:100E3000CE0B182F0800CC200B1D1C2F0800FF30F4
:100E4000E8006808E6007E26A9266A26CF26053037
:100E5000E90048081E02031C312FE90B292FE80B7B
:040E6000212F080036
:100F200082070000CD29D929E129E129F529072ADD
:100F3000192A252A2D2A372AF22CF22CF22CF22CEF
:100F4000F22CF22C462A4B2AF22CF22CF22CF22C08
:100F5000F22CF22CF22CF22C512AF22CF22C5E2ADA
:100F6000F22CF22CF22CF22C852A922A9F2AAA2A01
:100F7000B52AC02ACB2AD62AE62A2C2B5B2B662B35
:100F80007F2B862BF22CF22C8D2BAC2BBF2BF22C33
:100F9000D42BF22CE72BF22CF82B122C2C2C342CEB
:100FA000422C4E2C5A2C662C722C7E2C8A2C962C81
:100FB000A22CB02CBC2CC82CD42CDE2CE82CF22C6F
:020FC000080027
:1010000008308A005D088207003400340034322D35
:101010004E2D642DAA2DAB2DAC2DAD2DD22DD92D5D
:1010200008308A005D088207003400340034E32D64
:10103000012E5B2E5C2EE62EE72EE82ED22DEA2E18
:1010400008308A005D088207003400340034322DF5
:101050005D2D642D5D2D642D5D2DCA2D5D2DFF341C
:1010600008308A005D088207003400340034322DD5
:10107000562D642D562D642D562DC02D562DFF3422
:1010800008308A005D0882070034003400340134DF
:10109000083401340434013404340134023401349A
:1010A0000234023408308A005D08820700340034BC
:1010B0000034013404340134043401340434013480
:1010C00001340134023402342E2908308A005D08CC
:1010D0008207003400340034F12A112B362B432BC5
:1010E000902B912B922B932BB72B08308A005D0805
:1010F0008207003400340034CB2BD12BD22BD32BDE
:10110000D42BD52BDB2BDC2BE32B08308A005D089E
:101110008207003400340034D92CEE2C062D0D2D1E
:101120002C2D2D2D2E2D2F2D312D08308A005D08D0
:101130008207003400340034592C7C2CA12CAE2CB6
:10114000AF2CB02CB12CB22CC62C08308A005D0814
:101150008207003400340034EE2B0A2C1C2C1D2C8A
:0A116000352C362C372C452C462C7C
:1012000002293322BD08031D0829BC0803190E2931
:101210000130BC0203180129BD02012908000D227A
:101220005F21080020225F2108000D225F210800B5
:101230008A110A168E218A150A12871287118A11BD
:101240000A12A9268A150A127908BD007808BC007E
:1012500021303D0603192D29002108008A110A16A4
:101260008E218A150A12871287118A110A12A9265D
:101270008A150A127908BD007808BC0008008A1196
:101280000A168E218A150A12871287118A110A12EC
:10129000A9268A150A12C121A121BD017808BC0026
:1012A000002108008A110A168E218A150A12871257
:1012B00087118A110A12CF268A150A120800BA016C
:1012C000BB018A110A1695218A150A128715871102
:1012D0000830CF00871587110310871A0314BA0C42
:1012E000CF0B6A290630CF00871587110310871AA4
:1012F0000314BB0CCF0B7429BB0CBB0C87158711D7
:101300008A110A168E218A150A120800871287157B
:1013100087110830CF008716B80C031C8712871579
:101320008711CF0B8B290630CF008716B90C031C11
:10133000871287158711CF0B95298712871587117B
:1013400008003908C6003808C500FF30B900B800E9
:1013500086214608B9004508B80008000130F700AA
:10136000B7290230F700B7290430F700B7298A11EE
:101370000A12CC208A150A120B1DBC29F70BB729BB
:101380000800871287158711871287158711871222
:10139000871587118712871587118712871587117F
:1013A00087128715871108008716871587118712FE
:1013B000871587118712871587118712871587115F
:1013C00087128715871187128715871108008712E2
:1013D000871587118716871587118712871587113B
:1013E000871287158711871287158711871287152E
:1013F00087110800871687158711871687158711AB
:10140000871287158711871287158711871287150D
:101410008711871287158711080087128715871192
:1014200087128715871187168715871187128715E9
:101430008711871287158711871287158711080072
:1014400087168715871187128715871187168715C5
:1014500087118712871587118712871587118712C1
:10146000871587110800871287158711871687153A
:10147000871187168715871187128715871187129D
:10148000871587118712871587110800871687151A
:101490008711871687158711871687158711871279
:1014A000871587118712871587118712871587116E
:1014B00008008712871587118712871587118712F1
:1014C000871587118716871587118712871587114A
:1014D00087128715871108008716871587118712CD
:1014E000871587118712871587118716871587112A
:1014F00087128715871187128715871108008712B1
:101500008715871187168715871187128715871109
:1015100087168715871187128715871187128715F8
:101520008711080087168715871187168715871179
:1015300087128715871187168715871187128715D8
:101540008711871287158711080087128715871161
:1015500087168715871187168715871187168715B0
:101560008711871287158711871287158711080041
:10157000871287158711871287158711871287159C
:101580008711871687158711871687158711871288
:101590008715871108008716871587118716871505
:1015A0008711871687158711871287158711871668
:1015B00087158711871287158711080087168715E9
:1015C0008711871687158711871687158711871644
:1015D0008715871187168715871187128715871139
:1015E00008008A110A166D21B8006D21B9008A150C
:1015F0000A12E721862101305F0203190C2B8A11A0
:101600000A126E268A150A1276301E02031C0C2B53
:10161000B822B421C001102B5922B421B421C00139
:1016200008008A110A166D21B8006D21B9008A15CB
:101630000A12E7218621C00A49084006031D352BFE
:10164000DF08031D312B8A110A126E268A150A1231
:1016500076301E02031C312BB822AE21CB22C001F2
:10166000352B5922B421B421C00108008A110A1671
:101670006D21B8006D21B9008A150A12E721862173
:101680005922B4210800DF0803197C2B472B522173
:10169000AE21F901F8011821FF30B800B900E721A7
:1016A00086215922B121B121CB220830C6008A11EE
:1016B0000A166D21B8006D21B9008A150A12E721BA
:1016C00086210330C50033228A110A166D21B80025
:1016D0006D21B9008A150A12E7218621C50B632BFB
:1016E000B822B121B121CB223322C60B572BFF01E7
:1016F000FE01FD01FC018F2B8A110A166D21B80035
:101700006D21B9008A150A12E7218621C00A04302A
:101710004006031D8F2BB822B121CB22C001080047
:10172000362B432B362B8A110A166D21B8006D21FA
:10173000B9008A150A12E7218621C00A8A110A1601
:1017400050218A150A128A150A1233228A150A12A2
:101750008A110A166D21B8006D21B9008A150A1286
:10176000E72186215922AE21A522C00108008A1155
:101770000A166D21B8006D21B9008A150A12E721F9
:101780008621C00AB822B121A5228A110A12D020CE
:101790008A150A120800E72186215922B421B421B2
:1017A0000800CB2BCB2BCB2BCB2BE721862159222F
:1017B000B121CB220800CB2BE721862159225922C7
:1017C000AE21A5220800E7218621B822B121A52259
:1017D0008A110A12D0208A150A1208008A110A16E4
:1017E0006D21B8006D21B9008A150A12E721862102
:1017F000DF08031D072C8A110A126E268A150A12A9
:1018000076301E02031C072CB822B421092C592261
:10181000B42108008A110A166D21B8006D21B900A3
:101820008A150A12E7218621B822AE21CB221B2C71
:101830005922B421B42108000A2CFF30B800B900A5
:10184000E72186215922B121B121CB228A110A1622
:101850006D21B8006D21B9008A150A12E721862191
:10186000B822B121B121CB2208000A2C1D2C8A11EB
:101870000A166D21B8006D21B9008A150A12E721F8
:1018800086215922B421B42108000A2C8A110A1693
:101890006D21B8006D21B9008A150A12E721862151
:1018A000B822B121A5228A110A12D0208A150A1263
:1018B00008008A110A166D21B8006D21B9008A1539
:1018C0000A12E7218621C00A4A084006031D7B2C24
:1018D000DF08031D782C8A110A126E268A150A1257
:1018E00076301E02031C782CB822B421C0017B2C58
:1018F0005922B421C00108008A110A166D21B800CE
:101900006D21B9008A150A12E7218621C00A4A080A
:101910004006031DA02CDF08031D9C2C8A110A120F
:101920006E268A150A1273301E02031C9C2CB822E4
:10193000AE21CB22C001A02C5922B421B421C00178
:1019400008008A110A166D21B8006D21B9008A15A8
:101950000A12E72186215922B4210800432BA12C29
:10196000AE2CA12C8A110A166D21B8006D21B90088
:101970008A150A12E7218621C00A4A084006031D7B
:10198000C52C5922AE21A522C00108008A110A16D1
:101990006D21B8006D21B9008A150A12E721862150
:1019A000B822B121A5228A110A12D0208A150A1262
:1019B0000800FA218621DF08031DEA2C8A110A1289
:1019C0006E268A150A1276301E02031CEA2CB822F3
:1019D000B421EC2C5922B42133220800FA218621AB
:1019E000DF08031D012D8A110A126E268A150A12BC
:1019F00076301E02031C012DB822B421B421CB2263
:101A0000042D5922B421B42133220800FA21862161
:101A10005922B421B42133220800FA218621DF089B
:101A2000031D202D8A110A126E268A150A1276309D
:101A30001E02031C202DB822B421B421CB222A2D52
:101A40005922B121B121B121B121CB22B822B1213A
:101A5000B121CB2233220800062D0D2D062D003496
:101A60000800FF342030F9000730F8003F210F2133
:101A7000BB123B133B08B9003A08B800CB235221F4
:101A80002030F9000730F8003F21D42146225922A6
:101A9000B421B421D421462252210800F801F901D1
:101AA0003F21DE22B421B421522108006C22B4214E
:101AB000B4215922B421B42108009222B421B421C6
:101AC0005922B421B421080018210430C500FF3088
:101AD000C6003322C60B692DC50B672D3322332276
:101AE000332215213A08C2003B08C30052213F218E
:101AF0000F2143133B1A4317C313BB1AC317C1214A
:101B0000A1216C22B421B4219222B421B42152210A
:101B100018210430C500FF30C6003322C60B8D2DBE
:101B2000C50B8B2D3322332233224208B8004308E1
:101B3000B9003E2352213F210F213B12431B3B168C
:101B4000BB12C31BBB163A08B8003B08B900D2232E
:101B5000522108004E2D642D4E2D2030F900073003
:101B6000F8003F21E721A1216C22B421B421B42146
:101B7000B4219222B421B421B421B421522108000D
:101B80001821E721A1216C22B421B421B421B42170
:101B90005221080018219222B421B421B421B42189
:101BA00052210800F801F9013F216C22B421522191
:101BB00008003F21C121A1216C22B421B121B4210F
:101BC000B12152210800F801F90118216208C4006E
:101BD0006308C500EC2D3322FF30B800B900E721BF
:101BE00086215922B421C408031DF92DC508031903
:101BF000FF2D0130C5020318EB2DC402EB2D52213D
:101C000008000330F6006108C4006208C5006308DC
:101C1000C6000310C40CC50CC60CF60B092EF90146
:101C2000F80118210830F600FF30B800B900E721AC
:101C30008621F60B1C2E1E2E3322142E5922B4217F
:101C4000B421C408031D2A2EC508031D2A2EC60868
:101C50000319352E0130C6020318332EC5020318AE
:101C6000332EC402332E3322122EC1210430C6007B
:101C7000FF30B800B900E72186215922B421B421F0
:101C8000C60B432E452E3322382E3322FF30B800A8
:101C9000B900E72186215922B421B421332233220D
:101CA0003322FF30B800B900E72186215922B42140
:101CB000B42152210800642D8026C7266026080022
:101CC000F801F9013F21FF30B800B900E721862172
:101CD0005922B121B121CB220230C5000430C60007
:101CE0003322FF30B800B900E7218621C60B702EE1
:101CF000B822B121B121CB22C50B6E2E5221080092
:101D00000530F6006108C4006208C5006308C6001B
:101D10000310C40CC50CC60CF60B882EF901F80193
:101D20001821FF30B800B900E72186212030CB0010
:101D30000430F6005922B121CB22A12E0430F60046
:101D40003322FF30B800B900E7218621CB03F60B20
:101D5000A02EB822B121B121CB22CB080319B12E7C
:101D60009E2EC408031DBA2EC508031DBA2EC60830
:101D70000319E42E0130C6020318C32EC50203184E
:101D8000C32EC402C32E3322962E52210800B12145
:101D9000B121F901F8012E21FF30B800B900FA2174
:101DA0008621C6015922B121B121CB22FF30B800D2
:101DB000B900FA218621B822B121B121B121B12186
:101DC000CB223322C60BD22E52210800642D5C2E6A
:061DD000AD2DD22DFF3401
:1020000083171030840002308000840A063080007C
:10201000840A0530800008008317103084000130E6
:1020200080000800F1128A150A1240208A110A164F
:10203000C900C0018A150A1218218A110A165021F6
:10204000003A03192E288A150A1265208A110A16E9
:102050008A150A1233228A110A161F288A150A12B3
:1020600052218A110A160800F1128A150A126420F8
:102070008A110A165021003A031949286D21B80027
:102080008A150A1285208A110A16BC0F3A28BD0A41
:102090003A288A150A1252218A110A160800F112EA
:1020A000C0018A150A1252208A110A16CA008A151E
:1020B0000A123F218A110A165021003A03196B288F
:1020C0008A150A1295208A110A168A150A123322D5
:1020D0008A110A165C288A150A1252218A110A16D8
:1020E0000800F1128A150A123F218A110A1650219E
:1020F000003A03198C286D21B8006D21B9008A15AA
:102100000A1275208A110A16BC0ABC0A8A150A121C
:1021100033228A110A1677288A150A1252218A1147
:102120000A160800F112C0018A150A123F218A110D
:102130000A165021003A0319A8288A150A12A52068
:102140008A110A168A150A1233228A110A16992848
:102150008A150A1252218A110A160800F1128A15EC
:102160000A1218218A110A165021003A0319CD28A3
:102170008A150A1215218A110A163A088A110A12BA
:10218000D9253B088A110A12D9258A110A168A15FF
:102190000A1233228A110A16B4288A150A12522109
:1021A0008A110A160800F1128A150A1264208A118F
:1021B0000A165021003A0319ED288A150A12122135
:1021C0008A110A163A0873218A150A1233228A11D3
:1021D0000A16BC0FD928BD0AD9288A150A1252211D
:1021E0008A110A160800F1128A150A123F218A1173
:1021F0000A165021003A03190C298A150A121521D2
:102200008A110A163A0873213B0873218A150A12AB
:1022100033228A110A16F9288A150A1252218A11C4
:102220000A160800F1128A150A123F218A110A16AD
:102230005021003A03192B298A150A120F218A11FD
:102240000A163A0873213B0873218A150A123322B1
:102250008A110A1618298A150A1252218A110A1699
:102260000800F1128A150A123F218A110A1650211C
:10227000003A03194A298A150A1215218A110A16E9
:102280003A0873213B0873218A150A1233228A11F6
:102290000A1637298A150A1252218A110A160800CD
:1022A0008A110A16FF08031D5E29FE08031D5E2918
:1022B000FD08031D5E29FC08031900340130FC02EF
:1022C00003186929FD0203186929FE020318692908
:1022D000FF02FF308A110A1608008A110A12E1254E
:1022E0008A110A1608008A110A12D9258A110A16BB
:1022F00008008A110A126E268A110A1676301E020A
:10230000031C85298A150A1200288A150A1210282A
:102310008A150A1230288A150A1220288A110A12F0
:10232000E726F9268A110A1608008A110A12F026F1
:102330008A110A1608008A150A1262288A150A12DA
:1023400063288A150A1250288A150A1251288A1100
:102350000A1608000130C10008000230C100080060
:102360000230C100080083120313BF21C700CF2130
:10237000C8008A110A121F278A110A16DF29113094
:102380008A005D0882070034003400345E345E3415
:102390005E345E345E345E345E34A0348A34113090
:1023A0008A005D088207003400340034A934A9345F
:1023B000A934A934A934A934A934A634A93408000D
:0223C0000034E7
:103000000313831600309400831294120800831275
:1030100003130130580603194628023058060319D5
:10302000522803305806031959280430580603194A
:103030006B280930580603197D280A3058060319F1
:103040008F280C3058060319A1280D305806031993
:10305000DF280E30580603191929183058060319AD
:10306000262919305806031933291A30580603192E
:1030700035291B305806031937291C305806031907
:1030800038291D30580603194A2908005C21711897
:103090005128CF21831710308400590880008312F3
:1030A000031308005C21711858280330D6009921B9
:1030B00008005C2171186A288A110A16A121D6001D
:1030C0008A150A16A3218A110A16A421D6008A1588
:1030D0000A16B92108005C2171187C288A110A1689
:1030E000A121D6008A150A16A3218A110A16A42145
:1030F000D6008A150A16B92108005C2171188E289D
:103100008A110A169B21D6008A150A16A3218A1154
:103110000A169E21D6008A150A16B92108005C21DC
:103120007118A0288A110A169B21D6008A150A1642
:10313000A3218A110A169E21D6008A150A16B921E2
:103140000800F110831203137C08DA00EB21F11957
:10315000F1147D08DA00EB21F119F1147E08DA0090
:10316000EB21F119F1147808DA00EB21F119F114CF
:103170007908DA00EB21F119F1147A08DA00EB2171
:10318000F119F114CC288A110A12E1258A150A16C0
:10319000DA00EB21F119F114FE08031DD528FD0812
:1031A000031DD528FC080319DE280130FC02031892
:1031B000C328FD020318C328FE02C32808005C21AF
:1031C000711818298A110A169E21D6008A150A1626
:1031D0008317103084008001840A8001840A8001F2
:1031E000840A80019921831710308400840A840A9C
:1031F000840A0008D700103084000008840A840A7A
:10320000840A800010308400570880008317103033
:103210008400840A840A0008D70010308400840ADD
:103220000008840A800010308400840A5708800057
:1032300008005C21711825297808DA00EB2179084B
:10324000DA00EB217A08DA00EB2108005C21711822
:1032500032297808DA00EB217C08DA00EB217D08BE
:10326000DA00EB2108005C2108005C21080008005E
:103270005C2171188E288A110A16E021D6008A1561
:103280000A16A3218A110A16E021D6008A150A1609
:10329000B92108005C217118A0288A110A16E021C2
:1032A000D6008A150A16A3218A110A16E021D60033
:1032B0008A150A16B921080071105808DA00EB21A6
:1032C000FF30D900CF2159085A02031D7114D908C3
:1032D000031D6C297114CF2108008A110A16502190
:1032E0008A150A16003A031983294108D600CF210E
:1032F000711A832959088A110A12D9258A150A16C2
:10330000D60B77296D2908008A110A1650218A15D3
:103310000A16003A031998294108D6008A110A12A0
:10332000E1258A150A16DA00EB21D60B8E298429AD
:103330000800831710308400CF2159088000840AC8
:10334000D60B9C2908007808DA00EB21D603031974
:10335000B8297908DA00EB21D6030319B8297A08CD
:10336000DA00EB21D6030319B8297B08DA00EB2138
:1033700008007C08DA00EB21D6030319CE297D086A
:10338000DA00EB21D6030319CE297E08DA00EB21FF
:10339000D6030319CE297F08DA00EB210800930138
:1033A0000622F119E22971128A110A12F0268A15F1
:1033B0000A162530940094168C118C1DDD291308F3
:1033C000D900E329711687128A110A12E72694128E
:1033D0008A150A1608000622F119F72925309400EB
:1033E00094168C115A0893008C1DF429F7298A1120
:1033F0000A12D4208A150A160B1DFC2987128A117D
:103400000A12E72694128A150A1608008A110A126F
:10341000012787128A110A12E7268A150A16F11166
:10342000871D102A8A110A12D0208A150A160B1D30
:0C343000172A8716F11187191B2A0800C3
:04343C000034003424
:1038000083120313FB308605083086041030BE0097
:1038100020308400B02580003C302002031D0A2C9B
:10382000840ABE0B0A2CC3010C30BE002130840078
:103830000008C307840ABE0B182C0A30BE002530CE
:1038400084000008C1258000840ABE0B212C2808B2
:10385000B900270EB9042608B800250EB8042C08B4
:10386000BD002B0EBD042A08BC00290EBC0438087C
:10387000BA003908BB003D08BB07031C402CBA0A3C
:103880003C08BA073C302002031DBB2C3E302F02FF
:10389000031DBB2C2E08F5002D0EF5044308750200
:1038A000031DBE2C1B303A020319592C031C602C3B
:1038B000C12CFF303B020319602C0318C12C602C73
:1038C000003038020319672C03186D2CC12C04300A
:1038D000390203196D2C031CC12CC724B025A0008C
:1038E0007B302002031DBB2CC3013808F4003908CB
:1038F000F300F501F6010430BE0020308400B0254D
:10390000C307C1258000840ABE0B7F2C2308F60064
:10391000220EF6042108F500200EF504FF24000015
:103920000000000000000000000000000000000097
:10393000F30A0319F40A3A087402031D792C3B08B0
:103940007302031D792CB025C125A000B025C12527
:10395000A100200EA10443082102031DBE2CB025A6
:10396000A0007D302002031DBB2C83120313F7300F
:103970008605C724BA2C3130D824692D3430D82498
:10398000692D3630D824692D3730D824692D5B3025
:10399000AA253030AA253830AA253130AA25303062
:1039A000AA254330AA253930AA255D30AA2508006A
:1039B000F500B025A0007D3020020319E42C3E3034
:1039C00020020319E42CD92C5B30AA253030AA251B
:1039D0004130AA253030AA253030AA253030AA251A
:1039E0007508AA253330AA25750AAA255D30AA25AF
:1039F00083120313F730860504308604080003178A
:103A0000831273088D0074088F0075088C00760887
:103A10008E0083168C170C158B1355308D00AA3031
:103A20008D008C14000000000C1103138312080099
:103A30000317831273088D0074088F0083168C1788
:103A40000C140000000083120C08F7000E08F800A8
:103A5000031308008312031386168316403099005F
:103A6000243098008312903098001A081A087010B9
:103A70000800831203138C1A472D81010B11861243
:103A80008C1A472D7018402D0B1D402D492D1A08FA
:103A9000512D18194F2D98184F2D0301512D181223
:103AA00018168616BF01BF0B532DBF010800031364
:103AB0008312061A592D8316981C5C2D83129900C7
:103AC000080083120313D1256625692D2A25E925CF
:103AD00008007010B025F900553079020319812DC6
:103AE000563079020319922D5A3079020319962D16
:103AF000503079020319A42D463079020319A72DFD
:103B0000692D7014F01C852D872D18128A2D8316AF
:103B1000091283128312031306117530AA258A0134
:103B20001030820070147630AA25002C7014831295
:103B3000031306110130AA250130AA250130AA2558
:103B40000330AA257010692D86150611A62D0615BD
:103B50008611A92DF01CAE2D5725AF2D0526080086
:103B6000701CB92DF01CB72DB52D3925C02DF125B0
:103B7000C02DF018BC2DBE2DF010B72DF014B52DB2
:103B80000800FA00F9000F30F90547307A020318EF
:103B9000CF2D41307A02031CCF2D0930F907790867
:103BA0000800031383160B30850010308600903018
:103BB00087001730890004309F008312033087008C
:103BC00000308600103085008316D63081008312C5
:103BD000080003138316173089008312031306109D
:103BE0000800831203133D3081000B110614831665
:103BF000891B002E7018F72D0B1DF72D0301032EC6
:103C000083120610080806100800831203138800A8
:0E3C100006148316091B0A2E831206100800E4
:02400E003A3F37
:00000001FF
